:020000040800F2
:1000000000C00020F9020008211800082518000887
:10001000291800082D1800083118000800000000F9
:10002000000000000000000000000000351800087B
:1000300039180008000000003D18000841180008A9
:10004000F5140008F5140008F5140008F51400086C
:10005000F5140008F5140008F5140008F51400085C
:10006000F5140008F5140008F5140008F51400084C
:10007000F5140008F5140008F5140008F51400083C
:10008000F5140008F5140008F5140008F51400082C
:10009000F5140008F5140008F5140008F51400081C
:1000A000F5140008F5140008F5140008F51400080C
:1000B000F5140008F5140008F5140008F5140008FC
:1000C000F5140008F5140008F5140008F5140008EC
:1000D000F5140008F5140008F5140008F5140008DC
:1000E000F5140008F5140008F5140008F5140008CC
:1000F000F5140008F5140008F5140008F5140008BC
:10010000F5140008F5140008F5140008F5140008AB
:10011000F5140008F5140008F5140008F51400089B
:10012000F5140008F5140008F5140008F51400088B
:1001300000000000000000000000000000000000BF
:1001400000000000000000000000000000000000AF
:10015000000000000000000000000000000000009F
:10016000000000000000000000000000000000008F
:10017000000000000000000000000000000000007F
:10018000000000000000000000000000000000006F
:10019000000000000000000000000000000000005F
:1001A000000000000000000000000000000000004F
:1001B000000000000000000000000000000000003F
:1001C000000000000000000000000000000000002F
:1001D000000000000000000000000000000000001F
:1001E0005FF8E0F100B583B001F074F9304B314AAB
:1001F0001360314A1360314B314A03E011681960D2
:10020000043304322F498B42F8D32A4B1A682E4B01
:100210009A4204D1284B1A682C4B9A4200D0FEE730
:10022000234B2B4A13602B4A13602B4B02E0002216
:100230001A600433294A9342F9D3254B1B6813B93A
:10024000244B1B6803B1FEE701F050F9694601A891
:1002500001F038F9224C234B1C1BA410002504E0AC
:100260001F4B53F8253098470135AC42F8DC1E4C43
:100270001E4B1C1BA410002504E01B4B53F825301B
:1002800098470135AC42F8DC0099019801F042FA38
:100290000546174C174B1C1BA41004E0013C144BE3
:1002A00053F824309847002CF8DC284601F008F970
:1002B000BABADECA000000201000002000000020B2
:1002C000981A000814000020785634123254769898
:1002D00014000020BC01002014000020C0010020F8
:1002E0009403000894030008940300089403000892
:1002F000940300089403000808B5FFF773FF00BFDC
:1003000000BEFEE71EF0040F0CBFEFF30880EFF312
:1003100009807146124A104700BEFEE700BEFEE7A4
:100320001EF0040F0CBFEFF30880EFF30980714655
:100330000C4A104700BEFEE71EF0040F0CBFEFF39F
:100340000880EFF309807146074A104700BEFEE7B8
:1003500000BEFEE700BEFEE700BEFEE770470000FD
:0C03600019030008350300084D030008D5
:10036C00981A00080000002014000020981A0008B9
:10037C00000000000000000014000020C00100205C
:08038C00000000000000000069
:1003940010B5044600F0C4FF064BA3FB00308009EF
:1003A40000F098F8002221464FF0FF3000F050F89A
:1003B400002010BDD34D621008B5074A136843F0FE
:1003C40010031360032000F025F80020FFF7E0FF7E
:1003D40001F0B0F9002008BD00200240024A136871
:1003E40001331360704700BF18000020014B1868E8
:1003F400704700BF1800002010B582B00190FFF7CD
:10040400F5FF0446FFF7F2FF001B019B9842F9D366
:1004140002B010BD10B50446C31E042B03D9BA2183
:10042400094801F085F9094AD36823F4E0631B0401
:100434001B0C240204F4E064234343F0BF6343F43D
:100444000033D36010BD00BFB819000800ED00E010
:1004540070B504460E4615460F2A03D9D2211A4810
:1004640001F066F90F2E03D9D321174801F060F982
:10047400164BDA68C2F30222C2F10701042928BF2D
:100484000421131D062B01D9033A00E000220123A5
:1004940003FA01F101393140914003FA02F2013AC1
:1004A4002A400A43002C06DA04F00F041201D2B2E7
:1004B400074B1A5570BD1201D2B204F1604404F521
:1004C400614484F8002370BDB819000800ED00E011
:1004D40014ED00E00138B0F1807F0AD2064B586079
:1004E400F021064A82F823100020986007221A603F
:1004F40070470120704700BF10E000E000ED00E00D
:1005040010B50446042805D020B14FF4DF71084823
:1005140001F00EF9042C05D1064A136843F00403D4
:10052400136010BD034A136823F00403136010BD65
:10053400B819000810E000E008B501F0A3F908BDFF
:100544002DE9F04383B080460F46B54B98421BD04B
:1005540003F58063984217D003F58063984213D063
:1005640003F5806398420FD003F5806398420BD063
:1005740003F58063984207D003F58063984203D063
:10058400CF21A84801F0D4F83B881BB9D021A54855
:1005940001F0CEF87B68012B22D9112B20D0022B3D
:1005A4001ED0122B1CD0A04A934219D002F58012FF
:1005B400934215D002F58012934211D0A2F5F8129D
:1005C40093420DD002F58012934209D002F58012B5
:1005D400934205D0032B03D0D121924801F0A8F80F
:1005E4004FF000094E463FE10125B5403C682C40E0
:1005F400A54240F038818A4B98451BD003F58063AF
:10060400984517D003F58063984513D003F58063AC
:1006140098450FD003F5806398450BD003F58063AC
:10062400984507D003F58063984503D0DF217D48C2
:1006340001F07EF87B68122B49D00CD8022B3AD0FB
:1006440004D8002B4FD0012B1ED067E0032B60D0C1
:10065400112B24D062E0754A934244D008D8A2F505
:10066400801293423FD002F58032934256D13AE051
:100674006F4A934237D002F58032934233D0A2F5C9
:10068400801293424AD12EE0FB68013B022B03D92E
:10069400E721644801F04CF8D7F80C903EE0FB6881
:1006A400013B022B03D9EE215E4801F041F8FB68BF
:1006B40003F1040932E0FB68013B022B03D9F52165
:1006C400584801F035F8FB6803F1080926E0FB6897
:1006D400013B022B03D9FC21524801F029F8FB68A5
:1006E40003F10C091AE0BB68022B04D940F209118A
:1006F4004C4801F01DF8BB6873B1012B04D1C8F854
:1007040010504FF0080909E0C8F814504FF00809D8
:1007140004E04FF0000901E04FF00409FF2C01D878
:10072400404601E008F10400FF2C01D8B30002E0C8
:10073400A6F108039B0001680F229A4021EA0202F5
:1007440009FA03F3134303607B6813F0805F00F03E
:100754008A80384B9A6942F001029A619B6903F0DE
:1007640001030193019BB1088A1C334B53F8220007
:1007740006F003039B000F229A4020EA0200284A55
:10078400904515D002F58062904513D002F5806241
:10079400904511D002F5806290450FD002F5806239
:1007A40090450DD002F5806290450BD105220AE0F8
:1007B400002208E0012206E0022204E0032202E013
:1007C400042200E0062202FA03F3034302311A4A28
:1007D40042F821307B6813F4803F05D002F5806233
:1007E40013682343136004E0144A136823EA0403E0
:1007F40013607B6813F4003F04D0104A536823430A
:10080400536004E00D4A536823EA040353607B6891
:1008140013F4801F14D0094A93682343936014E0AF
:1008240000080140E8190008000011100000211020
:10083400000031100010024000000140000401409B
:100844000C4A936823EA040393607B6813F4001F43
:1008540004D0084AD3681C43D46004E0054AD36832
:1008640023EA0404D46001360F2E7FF6BDAE03B034
:10087400BDE8F0830004014070B5064615460C46F9
:1008840021B94FF4F271084800F052FF012D04D948
:1008940040F2E511044800F04BFF0DB1346170BD26
:1008A4002404346170BD00BFE819000838B504465B
:1008B4000D4621B94FF4FD71034800F039FFE1689A
:1008C4006940E16038BD00BFE819000830B583B065
:1008D400044620B94FF48771B94800F029FF236812
:1008E4003BB113F00F0F04D140F20F11B44800F0E4
:1008F4001FFF236813F0010F00F0A380636853B156
:10090400B3F5803F07D0B3F5A02F04D040F2151102
:10091400AB4800F00DFFAB4B5B6803F00C03042BFA
:100924000AD0A84B5B6803F00C03082B1BD1A54B22
:100934005B6813F4803F16D04FF4003393FAA3F3AB
:10094400A04B1A684FF4003393FAA3F3B3FA83F37A
:1009540003F01F0322FA03F313F0010F71D063684D
:10096400002B6ED11BE36368B3F5803F05D1954A34
:10097400136843F48033136026E063B903F18043C2
:1009840003F504331A6822F480321A601A6822F4D8
:1009940080221A6018E0B3F5A02F0CD103F1804334
:1009A400A3F53C331A6842F480221A601A6842F4B0
:1009B40080321A6008E0834B1A6822F480321A608D
:1009C4001A6822F480221A606368EBB1FFF70EFD07
:1009D400054605E0FFF70AFD401B642800F2E182AA
:1009E4004FF4003393FAA3F3764B1A684FF40033B1
:1009F40093FAA3F3B3FA83F303F01F0322FA03F386
:100A040013F0010FE6D01CE0FFF7F0FC054605E00B
:100A1400FFF7ECFC401B642800F2C5824FF400335E
:100A240093FAA3F3674B1A684FF4003393FAA3F3D2
:100A3400B3FA83F303F01F0322FA03F313F0010F55
:100A4400E6D1236813F0020F00F0A0802369012B84
:100A540004D940F249115A4800F06AFE63691F2B19
:100A640004D94FF4A571564800F062FE554B5B68FB
:100A740013F00C0F0AD0534B5B6803F00C03082BE4
:100A840027D1504B5B6813F4803F22D1022393FAA1
:100A9400A3F34C4B1A68022393FAA3F3B3FA83F338
:100AA40003F01F0322FA03F313F0010F03D02369A9
:100AB400012B40F07A824348036823F0F80163690C
:100AC400F82292FAA2F2B2FA82F293400B43036044
:100AD4005CE023699BB3012292FAA2F3B3FA83F395
:100AE4009B0003F1844303F584031A60FFF77EFC43
:100AF400054605E0FFF77AFC401B022800F2578206
:100B0400022393FAA3F32F4B1A68022393FAA3F355
:100B1400B3FA83F303F01F0322FA03F313F0010F74
:100B2400E8D02848036823F0F8016369F82292FAB0
:100B3400A2F2B2FA82F293400B43036026E001234F
:100B440093FAA3F3B3FA83F39B0003F1844303F50D
:100B5400840300221A60FFF749FC054605E0FFF70D
:100B640045FC401B022800F22482022393FAA3F3DB
:100B7400144B1A68022393FAA3F3B3FA83F303F032
:100B84001F0322FA03F313F0010FE8D1236813F0D3
:100B9400080F5CD0A369012B04D94FF4C571084830
:100BA40000F0C6FDA3696BB3012292FAA2F3B3FA73
:100BB40083F3054941F82320FFF718FC05460BE0B1
:100BC4002C1A00080010024080044242FFF70EFC79
:100BD400401B022800F2EF81022393FAA3F293FA56
:100BE400A3F2A44A526A93FAA3F3B3FA83F303F089
:100BF4001F0322FA03F313F0010FE7D00120FFF7DC
:100C0400FBFB24E0012393FAA3F3B3FA83F300215B
:100C1400994A42F82310FFF7E9FB054605E0FFF780
:100C2400E5FB401B022800F2C881022393FAA3F2D9
:100C340093FAA3F28F4A526A93FAA3F3B3FA83F3B3
:100C440003F01F0322FA03F313F0010FE7D1236823
:100C540013F0040F00F0AB80E368012B06D9052BD9
:100C640004D040F2B711854800F062FD814BDA6987
:100C740042F08052DA61DB6903F080530193019BF7
:100C84007F4A136843F480731360FFF7AFFB054694
:100C940005E0FFF7ABFB401B642800F29081784B22
:100CA4001B6813F4807FF4D0E368012B05D1714AEB
:100CB400136A43F00103136222E063B903F1804332
:100CC40003F504331A6A22F001021A621A6A22F046
:100CD40004021A6214E0052B09D1664B1A6A42F029
:100CE40004021A621A6A42F001021A6208E0614BB5
:100CF4001A6A22F001021A621A6A22F004021A62C3
:100D0400E36853B3FFF772FB054607E0FFF76EFB9A
:100D1400401B41F28833984200F25381022393FA34
:100D2400A3F293FAA3F3B3FA83F35B0943F0020348
:100D3400DBB2022B02D14F4B1A6A01E04D4B5A6AC7
:100D4400022393FAA3F3B3FA83F303F01F0322FA03
:100D540003F313F0010FD9D029E0FFF747FB054651
:100D640007E0FFF743FB401B41F28833984200F24F
:100D74002A81022393FAA3F293FAA3F3B3FA83F337
:100D84005B0943F00203DBB2022B02D1394B1A6A2E
:100D940001E0384B5A6A022393FAA3F3B3FA83F3BC
:100DA40003F01F0322FA03F313F0010FD9D1E3690F
:100DB400022B04D940F24721304800F0B9FCE36922
:100DC400002B00F002812B4A526802F00C02082A20
:100DD40000F0FD80022B40F0B780236A3BB1B3F5ED
:100DE400803F04D04FF41471244800F0A1FC636ADE
:100DF40073B3B3F5802F2BD0B3F5002F28D0B3F500
:100E0400402F25D0B3F5801F22D0B3F5A01F1FD0EB
:100E1400B3F5C01F1CD0B3F5E01F19D0B3F5001F04
:100E240016D0B3F5101F13D0B3F5201F10D0B3F5AF
:100E3400301F0DD0B3F5401F0AD0B3F5501F07D0B3
:100E4400B3F5601F04D040F251210C4800F070FC4F
:100E54004FF0807393FAA3F3B3FA83F39B0003F187
:100E6400844303F5840300221A60FFF7BFFA0546A2
:100E74000EE000BF00100240800442422C1A000819
:100E840000700040FFF7B2FA401B022800F2A18074
:100E94004FF0007393FAA3F3514B1A684FF00073A9
:100EA40093FAA3F3B3FA83F303F01F0322FA03F3D1
:100EB40013F0010FE6D1236AB3F5803F10D1A36884
:100EC4003BB1B3F5003F04D040F26721454800F040
:100ED4002FFC43494B6823F40032A36813434B604F
:100EE4003F48436823F47411236A626A13430B4333
:100EF40043604FF0807393FAA3F3B3FA83F39B0038
:100F040003F1844303F5840301221A60FFF76EFAA8
:100F1400044604E0FFF76AFA001B02285BD84FF08E
:100F2400007393FAA3F32E4B1A684FF0007393FAED
:100F3400A3F3B3FA83F303F01F0322FA03F313F0CA
:100F4400010FE7D0002049E04FF0807393FAA3F338
:100F5400B3FA83F39B0003F1844303F58403002273
:100F64001A60FFF743FA044604E0FFF73FFA001B58
:100F7400022832D84FF0007393FAA3F3184B1A687F
:100F84004FF0007393FAA3F3B3FA83F303F01F0350
:100F940022FA03F313F0010FE7D100201EE0012031
:100FA4001CE003201AE0032018E0012016E00320CF
:100FB40014E0032012E0032010E003200EE00320DD
:100FC4000CE003200AE0032008E0002006E00120F2
:100FD40004E0032002E0032000E0032003B030BD5E
:100FE400001002402C1A000830B486B01F4D02AC29
:100FF40028686968AA68EB680FC42B8AADF80430C6
:101004001B4B5B6803F00C02082A2AD103F470110D
:101014004FF4701292FAA2F2B2FA82F221FA02F2B8
:1010240006A90A4412F8102C13F4803F15D0104B73
:101034005B6803F400314FF4003393FAA3F3B3FA7B
:1010440083F321FA03F306A90B4413F8140C094B98
:10105400B3FBF0F000FB02F004E0074800FB02F0F1
:1010640000E0044806B030BC704700BF181A0008FE
:101074000010024000127A0000093D0070B50D46D0
:10108400044620B94FF42F71A04800F051FB2368A7
:1010940013F00F0F04D140F2BD219C4800F048FB2F
:1010A400022D04D940F2BE21984800F041FB984B30
:1010B4001B6803F007039D420BD9954A136823F07C
:1010C40007032B431360136803F007039D4240F0AA
:1010D4000D81236813F0020F1DD0A368A3B1802BE8
:1010E40012D0902B10D0A02B0ED0B02B0CD0C02B34
:1010F4000AD0D02B08D0E02B06D0F02B04D040F23D
:10110400D721824800F014FB82494B6823F0F00297
:10111400A36813434B60236813F0010F00F0818030
:101124006368022B04D940F2DE21784800F000FB0A
:101134006268012A13D14FF4003393FAA3F3754B79
:1011440019684FF4003393FAA3F3B3FA83F303F06B
:101154001F0321FA03F313F0010F28D1C8E0022A78
:1011640013D14FF0007393FAA3F36A4B19684FF04D
:10117400007393FAA3F3B3FA83F303F01F0321FA82
:1011840003F313F0010F12D1B4E0022393FAA3F393
:10119400604B1968022393FAA3F3B3FA83F303F0C1
:1011A4001F0321FA03F313F0010F00F0A58059493E
:1011B4004B6823F0030313434B60FFF717F906460C
:1011C4006368012B0FD107E0FFF710F9801B41F290
:1011D4008833984200F292804E4B5B6803F00C0314
:1011E400042BF1D11DE0022B16D107E0FFF7FEF826
:1011F400801B41F28833984200F28280454B5B6841
:1012040003F00C03082BF1D10BE0FFF7EFF8801B80
:1012140041F28833984275D83E4B5B6813F00C0F4B
:10122400F3D13B4B1B6803F007039D420AD2384AB3
:10123400136823F007032B431360136803F00703B9
:101244009D4261D1236813F0040F19D0E36883B180
:10125400B3F5806F0DD0B3F5A06F0AD0B3F5C06FAE
:1012640007D0B3F5E06F04D040F23231274800F0E4
:101274005FFA28494B6823F4E062E36813434B6048
:10128400236813F0080F1AD0236983B1B3F5806F74
:101294000DD0B3F5A06F0AD0B3F5C06F07D0B3F586
:1012A400E06F04D040F23931184800F041FA194A8D
:1012B400536823F46053216943EAC1035360FFF781
:1012C40093FE144B5B6803F0F002F02393FAA3F34C
:1012D400B3FA83F322FA03F30F4AD35CD8400F4BDB
:1012E40018600020FFF754F8002070BD012070BD85
:1012F400012070BD012070BD012070BD032070BDB0
:10130400032070BD032070BD012070BD2C1A00089D
:101314000020024000100240881A00080C0000203F
:10132400014B1868704700BF0C000020002800F033
:10133400BC8010B5044603685D4A93420BD0A2F505
:101344007842934207D002F58062934203D06B2126
:10135400584800F0EDF9636833B1B3F5827F03D0E8
:101364006C21544800F0E4F9A3684BB1B3F5806FE5
:1013740006D0B3F5004F03D06D214E4800F0D8F9E4
:10138400E368B3F5006F04D01BB16E21494800F047
:10139400CFF923692BB1022B03D06F21454800F00C
:1013A400C7F96369012B03D97021424800F0C0F9E1
:1013B400A369B3F5007F07D033B1B3F5802F03D011
:1013C40071213C4800F0B4F9E3698BB1082B0FD0CC
:1013D400102B0DD0182B0BD0202B09D0282B07D085
:1013E400302B05D0382B03D07221324800F0A0F9FD
:1013F400236A2BB1802B03D073212E4800F098F977
:10140400636A1BB174212B4800F092F9A36A33B1CB
:10141400B3F5005F03D07521264800F089F9E36A2B
:10142400013B4FF6FE72934203D97621214800F026
:101434007FF994F8513013F0FF0F02D1204600F0E9
:10144400C1F9022384F851302268136823F0400361
:10145400136021686268A3681A43E3681A43236926
:101464001A4363691A43A36903F400731343E269DB
:101474001343226A1343A26A1A430A602168638BE6
:1014840003F00402636A13434B602368E26A1A613F
:101494002268D36923F40063D3610020064B1870DB
:1014A4006065012384F8513010BD0120704700BFEE
:1014B40000300140581A00081C000020FEE700BF5D
:1014C40001230360014B0B60704700BF0400002040
:1014D40008B500F00FF8024B024A9A6008BD00BF3D
:1014E40000ED00E00000000808B500F029F808BD90
:1014F400FEE700000F4B1A6842F001021A605968B7
:101504000D4A0A405A601A6822F0847222F480322A
:101514001A601A6822F480221A605A6822F4FE02C1
:101524005A604FF41F029A604FF00062034B9A60B6
:10153400704700BF001002400000FFF800ED00E01B
:101544001F4B5B6803F00C03042B06D0082B08D058
:101554003BBB1C4A1C4B1A6026E01A4A1A4B1A6001
:1015640022E0174A53685268C3F38343023312F4E8
:10157400803F05D1154A02FB03F3134A136013E0BD
:101584000F4A526812F4003F05D0104A02FB03F3DD
:101594000D4A136008E00B4A02FB03F30A4A136086
:1015A40002E0084A084B1A60054B5B68C3F3031357
:1015B400074AD15C044A1368CB401360704700BFEC
:1015C4000010024000127A000C00002000093D00C7
:1015D400881A0008F0B587B01A4B9A6942F01002D5
:1015E4009A619A6902F010020092009A9A6942F094
:1015F40004029A619B6903F004030193019B124F57
:1016040000224FF400513846FFF736F90F4C002200
:101614000E212046FFF730F94FF4005302930126C0
:1016240003960225059502A93846FEF789FF0E2385
:1016340002930396059502A92046FEF781FF07B0A1
:10164400F0BD00BF0010024000100140000801403E
:1016540008B500F01BF9FEE708B50D480D4B036013
:101664004FF48273436000238360C360036143616A
:101674004FF4007282611822C26103624362836282
:101684000A23C362FFF752FE08B1FFF7E1FF08BD6A
:10169400240000200030014000B591B001230693DE
:1016A4004FF4803307930022089202220D920E9386
:1016B4004FF4E0130F9306A8FFF708F908B1FFF7FA
:1016C400C7FF0F23019302210291002303934FF4D8
:1016D40080620492059301A8FFF7D0FC08B1FFF7DC
:1016E400B7FFFFF71DFE094BA3FB00308009FEF78F
:1016F400F1FE0420FEF704FF002211464FF0FF30F4
:10170400FEF7A6FE11B05DF804FB00BFD34D6210D6
:1017140008B500F0AFF8FEF74FFEFFF7BDFFFFF787
:1017240059FFFFF799FF00F0B3F800F0A7F8FCE7C2
:10173400704700BF00B583B0204B9A6942F00102A4
:101744009A619B6903F001030193019B0320FEF757
:1017540061FE002211466FF00B00FEF779FE0022B5
:1017640011466FF00A00FEF773FE002211466FF077
:101774000900FEF76DFE002211466FF00400FEF72B
:1017840067FE002211466FF00300FEF761FE00229F
:1017940011466FF00100FEF75BFE002211464FF088
:1017A400FF30FEF755FE064A536823F0E06343F02A
:1017B4000073536003B05DF804FB00BF00100240E7
:1017C400000001400268134B9A4222D110B586B042
:1017D40003F560439A6942F480529A619B6903F469
:1017E40080530193019BA0230293022303930323B9
:1017F4000593094C02A92046FEF7A2FE402302935A
:1018040000230393049302A92046FEF799FE06B031
:1018140010BD70470030014000080140704700BF10
:10182400FEE700BFFEE700BFFEE700BFFEE700BF24
:10183400704700BF704700BF704700BF08B5FEF790
:10184400CDFDFEF779FE08BD08B54FF400510248FE
:10185400FFF72CF808BD00BF0010014008B54FF495
:101864007A7300221146024800F02EF808BD00BF2A
:101874004D18000808B500F00FF808BD08B500F0D1
:1018840043F808BD08B500F06BF808BD704700BF09
:1018940008B5FFF7E3FF08BD30B400230EE0094CA0
:1018A4009900CA18950060190022625142600272C0
:1018B400C2602846204402610133DBB20F2BEED90B
:1018C40030BC70477C000020F0B5002417E02746A8
:1018D40004EB8406B5000B4E3544ED686DB934460F
:1018E4004FEA870E0EEB0705AE00A519A2516B60F7
:1018F40000232B72E8602961F0BD0134E4B20F2C9F
:10190400E5D9F0BD7C00002070B5002422E004EB92
:1019140084029300114A1344DB68CBB104EB8402C4
:1019240093000E4A13441B7A93B1A10021448A0008
:101934000A4E1644013B3372F36830699847736862
:1019440033B904EB8405AB00044A13440022DA6083
:101954000134E4B20F2CDAD970BD00BF7C00002042
:1019640070B400231FE003EB83008200104802449C
:10197400D268B2B103EB830082000D48825852B999
:1019840004469A00D518A80025186E682650287AAF
:10199400411C297205E003EB83018800013A0449E4
:1019A4000A500133DBB20F2BDDD970BC704700BF86
:1019B4007C0000202E2E2F73797374656D2F737243
:1019C400632F73746D3332663178782F73746D338B
:1019D40032663178785F68616C5F636F72746578C2
:1019E4002E6300002E2E2F73797374656D2F73721E
:1019F400632F73746D3332663178782F73746D335B
:101A040032663178785F68616C5F6770696F2E63E6
:101A14000000000002030405060708090A0B0C0D68
:101A24000E0F1010010200002E2E2F7379737465AF
:101A34006D2F7372632F73746D3332663178782F20
:101A440073746D3332663178785F68616C5F72638A
:101A5400632E63002E2E2F73797374656D2F73724A
:101A6400632F73746D3332663178782F73746D33EA
:101A740032663178785F68616C5F7370695F65782E
:101A84002E630000000000000000000001020304B7
:041A94000607080930
:101A980078563412200000200000000000A24A04FA
:041AA80032547698A6
:04000005080001E509
:00000001FF
